:020000040800F2
:10000000001800203B5C0008E95B0008B15C0008B8
:10001000ED5B0008EF5B0008F15B000800000000EA
:10002000000000000000000000000000F35B00087A
:10003000F55B000800000000F75B0008350E0008C3
:10004000FB5B0008FD5B0008FF5B0008015C00082B
:10005000035C0008055C0008075C0008095C0008F8
:100060000B5C00080D5C00080F5C0008115C0008C8
:10007000135C0008155C0008175C0008195C000898
:100080001B5C00081D5C00081F5C0008215C000868
:10009000235C0008255C0008275C0008295C000838
:1000A0002B5C00082D5C00082F5C0008B90E0008CE
:1000B000335C0008355C0008375C0008395C0008D8
:1000C00082B0002301930093304A116880235B02C1
:1000D0000B431360110080229202A020C0010B6824
:1000E00013400093019B01330193009B002B02D12D
:1000F000019B8342F3D1254B1B689B0339D5244BCD
:1001000011221A60214A5368F0218B435360214B1E
:100110001B68102B2FD0042B32D01C4B5A685A600E
:100120001A4B5A685A605A681B490A405A60596803
:10013000882252030A435A601968802252040A43F3
:100140001A601900802292040B681342FCD00F4BF6
:100150005A6803218A435A605A6801390A435A602F
:1001600019000C224B681340082BFBD1074B0122CE
:100170001A6302B07047536840390B435360CFE7AE
:10018000024A536890210B435360C9E700100240B4
:0C01900000200240E4140020FF7FC0FFAC
:10019C00124B1B68002B0FD1104B32221A60104BE4
:1001AC001B68012B0ED90F4B1B68002B05D0013B94
:1001BC000C4A1360002B00D070470B4B802252006E
:1001CC009A61F9E7002B04D1074B802252049A6103
:1001DC00F2E7054B802252009A61EDE7581500209A
:0C01EC006015002064150020000400488D
:1001F80010B5054B1860002805D01C00FFF7CAFF92
:0C0208002368002BFAD110BD68150020FF
:1002140010B504F03DFC154B1A68D34301321BD0D2
:10022400FF22110019401A4217D0114A11601B0213
:100234001B0E16D00F4A13600E4B1A680E4B1A6031
:100244000E4B1968CA43FF23180088430C49086001
:10025400120C13400B4A136010BD054A0B211160A8
:10026400E5E7044B0A221A60E6E7C046006400088A
:100274007015002004150020C81400200464000830
:080284005C150020601500204C
:10028C0010B544490122CB681A42FCD1414B1B6981
:10029C001B0604D53F4B404A5A60404A5A603D4BBE
:1002AC001A6902210A431A613D4A5A611A693E31A0
:1002BC000A431A6119000122CB681A42FCD1354B52
:1002CC00DB689B0604D5334AD36820210B43D360EB
:1002DC00304B1A6902218A431A611A6901390A439F
:1002EC001A61304B1B68DB432D4A138029490122CC
:1002FC00CB681A42FCD1274BDB689B0604D5254AF8
:10030C00D36820210B43D360274B1B68DB43274A60
:10031C00138020490122CB681A42FCD11D4BDB68AB
:10032C009B0604D51B4AD36820210B43D360204B7A
:10033C001B68DB431F4A138016490122CB681A4203
:10034C00FCD1144BDB689B0604D5124AD3682021E0
:10035C000B43D360184B1B68DB43184A13800D49C1
:10036C000122CB681A42FCD10A4BDB689B0604D5F0
:10037C00084AD36820210B43D360064B1A6901212C
:10038C008A431A611A697F310A431A610A20FFF7FE
:10039C002DFF10BD0020024023016745AB89EFCD36
:1003AC000064000870150020041500200264000889
:1003BC005C15002004640008601500200664000829
:1003CC00F8B5C34B1C68631E012B00D915E2C1495B
:1003DC000122CB681A42FCD1BE4B1B691B0604D50B
:1003EC00BC4BBD4A5A60BD4A5A60BA4A13690221D5
:1003FC000B431361012C00D1C4E0B64BB84A5A61CF
:10040C00B44A136940210B43136111000122CB68DC
:10041C001A42FCD1AF4BDB689B0604D5AD4AD368BE
:10042C0020210B43D360AB4B1A6902218A431A611A
:10043C001A6901390A431A61013C63425C41644206
:10044C00A84B1C40A64B9C466444A74B1B6801332D
:10045C00DB4323809F490122CB681A42FCD19D4B80
:10046C00DB689B0604D59B4AD36820210B43D360E1
:10047C009E4B1B68DB43638096490122CB681A4272
:10048C00FCD1944BDB689B0604D5924AD36820219F
:10049C000B43D360964B1B68DB43A3808D49012231
:1004AC00CB681A42FCD18B4BDB689B0604D5894A7E
:1004BC00D36820210B43D3608E4B1B68DB43E38056
:1004CC0084490122CB681A42FCD1824BDB689B0623
:1004DC0004D5804AD36820210B43D360864B1B681C
:1004EC001B02864A12781343DB432381794901228C
:1004FC00CB681A42FCD1774BDB689B0604D5754A56
:10050C00D36820210B43D3607D4B1B68DB43638195
:10051C0070490122CB681A42FCD16E4BDB689B06FA
:10052C0004D56C4AD36820210B43D360754B1B68F0
:10053C001B02DB43A38167490122CB681A42FCD121
:10054C00644BDB689B0604D5624AD36820210B43BD
:10055C00D3606D4B1B68DB43E3815E490122CB68A2
:10056C001A42FCD15B4BDB689B0604D5594AD36815
:10057C0020210B43D36010346448564B01222025B4
:10058C00634E07E01300634A5A6139E704340430C0
:10059C00B04219D00168C9432180D9680A42FCD104
:1005AC00D9680D4202D0D9682943D9600168C94382
:1005BC00090C6180D9680A42FCD1D9680D42E5D09A
:1005CC00D9682943D960E1E7424B1A6901218A4372
:1005DC001A611A6901310A431A613D4B1C68012CDE
:1005EC002DD03C4B4C4A5A613A4A136940210B437B
:1005FC00136111000122CB681A42FCD1354BDB6828
:10060C009B0604D5334AD36820210B43D360314B6E
:10061C001A6902218A431A611A6901390A431A615B
:10062C00013C63425C4164422E4F27403A4B9C464E
:10063C0067443C00274B01222025384E07E0254B10
:10064C00374A5A61D0E704340430B04219D00168FB
:10065C00C9432180D9680A42FCD1D9680D4202D025
:10066C00D9682943D9600168C943090C6180D968EC
:10067C000A42FCD1D9680D42E5D0D9682943D9602A
:10068C00E1E780239B009C4667442648114B0122DE
:10069C002025254E03E004370430B04246D00168D3
:1006AC00C9433980D9680A42FCD1D9680D4202D0BD
:1006BC00D9682943D9604188C9437980D9680A42ED
:1006CC00FCD1D9680D42E6D0D9682943D960E2E75C
:1006DC005C1500200020024023016745AB89EFCD5B
:1006EC000074000800F4FFFF6015002004150020C2
:1006FC0048150020E4140020D8140020E014002039
:10070C00DC140020001500203815002004080020FF
:10071C00F40B00200068000800780008F40D00209D
:10072C00006C00080402002004040020334B1A69FA
:10073C0001218A431A611A6901310A431A61304B4B
:10074C001C68012C2CD02D4B2E4A5A612B4A136954
:10075C0040210B43136111000122CB681A42FCD1DA
:10076C00264BDB689B0604D5244AD36820210B4317
:10077C00D360224B1A6902218A431A611A69013922
:10078C000A431A61013C63425C4164421E4B1C40AB
:10079C001C4B9C466444194B012220251B4E07E040
:1007AC00164B1B4A5A61D1E704340430B04218D0BE
:1007BC000168C9432180D9680A42FCD1D9680D422D
:1007CC0002D0D9682943D9604188C9436180D9686E
:1007DC000A42FCD1D9680D42E6D0D9682943D960C8
:1007EC00E2E7064B1A6901218A431A611A697F31C3
:1007FC000A431A610A20FFF7F9FCF8BD00200240F9
:10080C005C150020007C000800F4FFFF04080020A9
:04081C000070000860
:10082000284A91698023DB010B4393619023DB0508
:100830001A6825490A401A601968A02292030A43DF
:100840001A605A6A21490A405A62596A882252003B
:100850000A435A621E4B1F4A13601F4A13601F4B04
:100860001B68392B29D01ED8132B28D0263B5A1EA3
:1008700093415B421A4A13401A4A944663441A4A07
:10088000938180239B025360002393602C33136079
:10089000136801210B431360144B1960144B802221
:1008A00012051A607047603B5A1E93415B42114A21
:1008B0001340114A94466344E1E7104BDFE7104BC5
:1008C000DDE7C04600100240FFFFEBFF0FF0FFFF27
:1008D00014110020501500204C1500207015002028
:1008E000BFFCFFFFE2040000003801406C1500204F
:1008F00000E100E019EEFFFF881300004103000053
:04090000C409000026
:100904000A498022CB691A42FCD080B2074B188571
:10091400074B1B68032B00D07047064B8022520400
:100924009A61054B04221A60F6E7C046003801407C
:0C0934006015002000040048641500203D
:10094000F0B5C64600B5494B1B68002B65D0013B8E
:100950005A4253415B42464C1C40464B9C466444C1
:100960002068C3436168CA430140013100D16EE091
:100970001904090C0139404801601B0CFF210B4090
:100980003E4803603E480360130C0B403D490B603A
:10099000012B04D0102B02D00B000121196012048E
:1009A000120C394B1A60A368DB439A05920F374942
:1009B0000A603F221A4036490A601B0C354A136010
:1009C000E368DE4325001035370C334B1F603F01D1
:1009D0002C4B1B6898461900380005F0A7FB2F4BDD
:1009E000186033041B0E7E2B01D901235B422C4A75
:1009F000136047452ED22B4A2B4908CDDB4308C252
:100A00008A42FAD1C023DB009C466444274A284826
:100A100008CCDB4308C28242FAD103F071FE1A4BC4
:100A20001B68002B07D09023DB051B8A5B0502D4D3
:100A3000154B00221A600D20FFF764FF01F0CCF97E
:100A4000114B1B68002B0AD180BCB846F0BD04F0E6
:100A500021F8E2E702F052FA02F0C6FACBE7013BD6
:100A6000144A136003F058FBEEE7C0465C15002003
:100A700000F4FFFF0074000860150020041500203A
:100A8000C8140020E414002048150020D8140020C9
:100A9000E0140020DC140020381500201C15002074
:100AA0000015002004080020F40D0020040200209E
:080AB00004080020FC140020E2
:100AB80070B5041E00DA9CE0092C00D893E0632C82
:100AC80000D881E0FA239B009C426ED3534B9C4292
:100AD8005AD9534B9C4248D9524B9C4236D9524B17
:100AE8009C4224D9514B9C4212D9514B9C4200D96B
:100AF80084E05049200005F015FB05004D49200011
:100B080005F075FA0C0028003030C0B2FFF7F6FE89
:100B18004949200005F006FB05004749200005F07B
:100B280066FA0C0028003030C0B2FFF7E7FE4349F0
:100B3800200005F0F7FA05004049200005F057FAB3
:100B48000C0028003030C0B2FFF7D8FE3C49200026
:100B580005F0E8FA05003A49200005F048FA0C00CB
:100B680028003030C0B2FFF7C9FE3649200005F032
:100B7800D9FA05003349200005F039FA0C0028009D
:100B88003030C0B2FFF7BAFEFA218900200005F024
:100B9800C9FA0500FA218900200005F028FA0C009E
:100BA80028003030C0B2FFF7A9FE6421200005F00C
:100BB800B9FA05006421200005F019FA0C00280094
:100BC8003030C0B2FFF79AFE0A21200005F0AAFAD9
:100BD80005000A21200005F00AFA0C002800303030
:100BE800C0B2FFF78BFE20003030C0B2FFF786FEA0
:100BF80070BD2D20FFF782FE64425DE71249200098
:100C080005F090FA05001049200005F0F0F90C00F5
:100C180028003030C0B2FFF771FE6AE70F270000E6
:100C28009F8601003F420F007F969800FFE0F50580
:100C3800FFC99A3B00E1F5058096980040420F00F5
:0C0C4800A08601001027000000CA9A3BA3
:100C540070B5484D484C02E06420FFF7CBFA474B8F
:100C64005969802292020A435A6159698022D20248
:100C74000A435A619021C90500260E60404B1E604C
:100C8400404ACA60DA60D9683F480140D9601A68AE
:100C940002401A601968802252020A431A608022B4
:100CA40052009A6101232B60FFF708FA374B1E604C
:100CB400374B1E60374B1E60374B0B221A60374B85
:100CC4001E600A23364A1360364A1360364B0322E9
:100CD4001A60364B364A1A602B685901C91A8900C2
:100CE400C918C900334B186805F01EFA013880236F
:100CF4005B0498420DD2304A50603048036A1B02AC
:100D04001B0AC02109060B430362002393600733C7
:100D140013603220FFF76EFA03F0F0FCFFF778FA65
:100D24000220FFF767FAFFF779FD0220FFF762FA66
:100D34000D20FFF7E5FD224804F0FBFF3120FFF70B
:100D4400DFFD2E20FFF7DCFD0B20FFF7B3FE1D486F
:100D540004F0EFFFFFF7F2FD03F038FD02F00AFAAA
:100D6400002800D178E72368002BF5D003F036FA89
:100D7400F2E7C046E4140020BC1400200010024036
:100D840000040048AAAAAAAAFFFFFCFF64150020D9
:100D94006815002054150020701500206C150020E3
:100DA40004150020C814002060150020F014002051
:100DB400A1B0B9120002002010E000E000ED00E054
:080DC400CC5C0008B0540008EB
:100DCC0010B5FFF7E5F9114B1B68114A12689342F5
:100DDC0019D05A1C0D490A601B7880200002184358
:100DEC000C4B1B689A420BD00B4B1B68012B06D982
:100DFC000A4B802252049A61094B04221A6010BDDE
:100E0C00084A0A60F0E70020F9E7C0464C150020BC
:100E1C0050150020FC010020601500200004004843
:080E2C006415002014110020E0
:100E3400194B1B68002B02D0013B174A1360174B58
:100E44001B68002B02D0013B144A1360144B1B682F
:100E5400002B02D0013B124A1360124B1B68002B7B
:100E640002D0013B0F4A13600F4B1B68002B02D0CA
:100E7400013B0D4A13600D4B1B68002B02DD013B47
:100E84000A4A13600A490A6853035A40530C5340F0
:100E94005A0153400B607047581500206815002014
:100EA4005415002010150020CC140020E814002054
:040EB400F014002016
:100EB80010B5114BDB699B0612D50F4B9B8C99B271
:100EC800FF221340022B0CD0042B12D00B4A1368BC
:100ED8001970136801331360094A1268934204D0E9
:100EE80010BD084BFD3A1A60F0E7044B064A1A6039
:100EF800F6E700F095FDF3E70038014050150020B3
:0C0F0800FC010020C01400201411002087
:100F1400024A202311680B431360704724150020F4
:100F2400064A1368043B1360054A0C32934204D208
:100F3400044A042311680B4313607047EC14002027
:080F4400881300202415002091
:100F4C00084B1A68111D1960074B6033994202D285
:100F5C00136853607047054A042311680B431360F0
:100F6C00F8E7C046EC14002088130020241500205C
:100F7C00044B19680A1F1068096811601B68186017
:080F8C007047C046EC14002080
:100F9400034A1368191D11601A1F12685A607047BA
:040FA400EC14002029
:100FA800074A1368190008390868043B1B680B6076
:100FB8001368191F1B680B60136818607047C046D8
:040FC800EC14002005
:100FCC00074A13681968181F006818601368181FFF
:100FDC00083B1B6803601368083B19607047C046E8
:040FEC00EC140020E1
:100FF0000C4B19680A680C4BCB1A9B109B1A042BDC
:1010000006D4002A0AD092008A1A13680B6070472F
:10101000064A042311680B431360F8E70439014BB7
:101020001960F4E7EC140020881300202415002038
:1010300030B5144B1A681168134BD31A9B105B1A06
:10104000042B19D4043A0F4B1A60012913D9012338
:101050005B1A9B009D580222521A9200094C236889
:1010600098589B18043B1860013904320029F6D1C6
:10107000044B1B681D6030BD044A042311680B43F8
:101080001360F8E7EC1400208813002024150020DA
:10109000F0B5144B1A681568134BD31A9B105B1BE1
:1010A000042B19D4043A17680E4B1A60012D12D97B
:1010B0006E1E0422524200211C00236898589B187F
:1010C00058600131043AB142F7D101235D1B054B51
:1010D0001B68AD00EF50F0BD044A042311680B43B8
:1010E0001360F8E7EC14002088130020241500207A
:1010F000054B1A68111F12680868844662440A602A
:0C1100001A68043A1A607047EC140020D2
:10110C00024B1A681368013313607047EC1400200B
:10111C00054B1A68111F12680868821A0A601A684F
:0C112C00043A1A607047C046EC14002022
:10113800024B1A681368013B13607047EC140020D7
:10114800044B1A681368002B00DB70475B4213607E
:08115800FBE7C046EC14002087
:1011600010B50F4B1B681A68D117501848401F283C
:1011700009DC191F0A4C2160002A0BDB0B000968EF
:101180009140196010BD074A8023DB0011680B43B2
:101190001360F7E7043B1A68C2401A60F2E7C046E2
:0811A000EC14002024150020CE
:1011A800054B1A68111F1268086802400A601A681D
:0C11B800043A1A607047C046EC14002096
:1011C400054B1A68111F1268086802430A601A68FE
:0C11D400043A1A607047C046EC1400207A
:1011E000054B1A68111F1268086842400A601A68A5
:0C11F000043A1A607047C046EC1400205E
:1011FC00024B1A681368DB4313607047EC14002031
:10120C00024B1A6813685B4213607047EC140020A1
:10121C00054B1A68111F1268086842430A601A6865
:0C122C00043A1A607047C046EC14002021
:1012380010B50B4B1C682168002909D0043C2068B4
:1012480004F052FF2060064A1368043B136010BD87
:10125800044A80231B0111680B431360F7E7C0465B
:08126800EC1400202415002005
:1012700010B50B4B1C68216800290AD0221F10688A
:10128000083C23685843064B1C6004F031FF206083
:1012900010BD044A80231B0111680B431360F7E75C
:0812A000EC14002024150020CD
:1012A80010B50B4B1C682168002909D0043C206844
:1012B80004F04CFF2160064A1368043B136010BD1C
:1012C800044A80231B0111680B431360F7E7C046EB
:0812D800EC1400202415002095
:1012E00070B50D4B1C682568002D0ED0043C266897
:1012F0002900300004F02EFF2160074B1C682900F4
:10130000300004F0F5FE206070BD044A80231B010C
:1013100011680B431360F7E7EC140020241500203C
:101320000B4B1B681A681F2A0BD8043B0121914004
:101330000A0019680A431A60054A1368043B1360DF
:101340007047044A8023DB0011680B431360F7E702
:08135000EC140020241500201C
:101358000B4B1B681A681F2A0AD8043B01219140CD
:101368001A688A431A60064A1368043B1360704778
:10137800044A8023DB0011680B431360F7E7C0467B
:08138800EC14002024150020E4
:101390000C4B1B681A681F2A09D8012191400A00CA
:1013A000191F0968114209D001221A6005E0064A96
:1013B0008023DB0011680B431360704700221A6022
:0C13C000FBE7C046EC14002024150020C0
:1013CC00034A1368191D1160024A12685A6070476B
:0813DC00EC140020F0140020C5
:1013E400064A1368191F1B6808681B1A58424341B0
:1013F4000B601368043B13607047C046EC14002074
:10140400064A1368191F1B6808681B1A581E834173
:101414000B601368043B13607047C046EC14002053
:10142400034B1A6811684B424B4113607047C04626
:04143400EC14002094
:10143800074B1A68131F012112681868904200DCD4
:1014480000211960024A1368043B13607047C046C4
:04145800EC14002070
:10145C0030B5074B1A68111F10680A68D217C40FF1
:10146C000D68854262410A601A68043A1A6030BD00
:04147C00EC1400204C
:10148000074B1A68131F012112681868904200DB8D
:1014900000211960024A1368043B13607047C0467C
:0414A000EC14002028
:1014A400064A1368191F1B68086884469C459B41BB
:1014B4005B420B601368043B13607047EC1400201C
:1014C40030B5074B1A68111F08681468C20FE51776
:1014D40084426A410A601A68043A1A6030BDC04600
:0414E400EC140020E4
:1014E800114B1A681368002B0CD0C82B0ADC1900A2
:1014F800C83107DB002B0CDD013B9B000B495B5817
:10150800136005E00A4A8023DB0011680B4313606F
:101518007047DB439B00111F086804495850083A7C
:10152800014B1A60F4E7C046EC140020F40D0020CB
:041538002415002056
:10153C00044B0A221A60044B1B68002B01D1034B8D
:10154C001A607047C81400202815002004150020CC
:10155C00044B10221A60044B1B68002B01D1034B67
:10156C001A607047C81400202815002004150020AC
:10157C0005490A681368043A0A60002B02D0013B43
:0C158C00002BFCD17047C046EC1400207E
:1015980004490B6864221868424303480260043B0C
:0C15A8000B607047EC140020CC140020F5
:1015B40010B5054B1C68221D1A60044B1868642181
:1015C40004F0B2FD606010BDEC140020CC140020C7
:1015D40030B5094B1B68013B08495B181B041C0C04
:1015E400074802681B0E15684B5513689C466144F6
:1015F4004C70043A026030BD34150020040200200F
:04160400EC140020C2
:10160800044B1A68111D1960034B1B68043B1B68C7
:0C16180053607047EC140020F414002014
:10162400024B1B681A68024B1A607047F4140020BE
:041634001815002065
:10163800064B1B681A68002A04D1054A126811680B
:10164800044A1160043B014A13607047EC140020FF
:08165800F41400201815002015
:10166000154B1B68154A19681160154A934218D921
:10167000144A1268022A07D0043B0F4A1360124A28
:101680001368013B136070470F4A11680F4A1268D4
:101690009142F1D10D4A002111600A4A03311160D3
:1016A000EAE7064B00221A60064B1B68022BEAD1C0
:1016B000044B03321A60E6E7F414002018150020EA
:1016C00018130020F80100200C15002044150020FC
:1016D000054B00221A605A609A6018000C300349CA
:1016E0000860DA607047C04688130020EC140020C0
:0C16F000014B03221A607047F801002033
:0C16FC00014B01221A607047F801002029
:0C170800014B00221A607047F80100201D
:1017140030B50D4B1C68221D1A600C490B685A1C0D
:101724000A60587800069A1C0A609A7812040243E8
:10173400D81C0860D87800021D1D0D601B79134366
:101744000343636030BDC046EC140020181500202C
:10175400054A1368191D116004490A68501C086081
:1017640052785A607047C046EC14002018150020C7
:10177400074B19680A1D1A60064A1368581C106042
:101784005A781201044B9B189B684B607047C04603
:0C179400EC1400201815002004080020B0
:1017A000074B1A68511C19600648036851780901F3
:1017B000054A521819689160043B03607047C0469F
:0C17C00018150020EC1400200408002084
:1017CC00074B1A68511C196051780902901C18605B
:1017DC0092781143802292050A431A607047C046E2
:0417EC0018150020AC
:1017F00010B5094B1868021D1A6008490B685A1C7D
:101800000A605A7812029C1C0C609B781A43802351
:101810009B051343436010BDF414002018150020ED
:10182000074B1A68511C196051780902901C186006
:1018300092781143802292050A431A607047C0468D
:041840001815002057
:1018440010B5094B1B681A68023A80239B051343A1
:101854001A78742A03D1013B044A136010BD034A69
:101864001360FFF7DBFFF9E7F414002018150020DC
:1018740010B50A4B1B681B68002B0CD0084A136870
:10188400043B1360074A136803331360034A136865
:10189400043B136010BDFFF7C1FFF7E7EC14002011
:0818A400F414002018150020C7
:1018AC0010B50A4B1B681B68002B0CD1084A136837
:1018BC00043B1360074A136803331360034A13682D
:1018CC00043B136010BDFFF7A5FFF7E7EC140020F5
:0818DC00F4140020181500208F
:1018E40010B5104B1A681100103119600E490B68BD
:1018F400180008380068D060181F006890601868E5
:1019040050600C3B0B6009480368591C016059780E
:1019140009029C1C04609B78194380239B050B439C
:10192400136110BDF4140020EC14002018150020DD
:10193400204B1B681A1F12681900083908680439FB
:101944000968521800291ADB904210DD043B1A6022
:10195400194B1A68511C196051780902901C1860BF
:1019640092781143802292050A431A607047103B13
:10197400104A1360104A136803331360F6E7904269
:1019840010DA043B1A600C4B1A68511C1960517828
:101994000902901C186092781143802292050A4330
:1019A4001A60E3E7103B034A1360034A13680333E6
:0C19B4001360DBE7F4140020181500207D
:1019C000024A1368043B13607047C046F4140020B9
:1019D000024A1368103B13607047C046F41400209D
:1019E00008490B681A6808480260043B0B60032A28
:1019F00000D87047054A8023DB0011680B43136051
:101A0000F7E7C046EC1400206015002024150020E4
:101A100010B5044C23681878FEF774FF2368043B64
:081A2000236010BDEC1400204E
:101A280010B50F4B1B68002B00D010BD2020FEF70F
:101A380065FF2D20FEF762FF3E20FEF75FFF442082
:101A4800FEF75CFF4220FEF759FF4720FEF756FFDE
:101A58002020FEF753FF024B01221A60E5E7C0463B
:041A6800F801002061
:101A6C0070B50A490A68561C0E6054783619002C59
:101A7C0009D00D002B685A1C2A605878FEF73CFFE1
:101A8C00013C002CF6D1014B1E6070BD18150020D6
:101A9C0010B5114B1B68002B12D0104B1B68002B80
:101AAC000ED00F4B1B68002B15D00E4A1368191D56
:101ABC0011600D4A12785A60094B00221A600AE034
:101ACC00FFF77EF90028FBD0064B1A68111D196030
:101ADC00FF231840506010BDF80100202015002095
:0C1AEC00C4140020EC140020741500202D
:101AF80010B50E4B1B68102B08D00D4B1B681868CF
:101B0800E0231B06C2180B4B9A420CD8084B1B68E3
:101B1800186804F0DDFA2020FEF7F0FE044A136886
:101B2800043B136010BDFEF7C3FFF4E7C8140020A0
:081B3800EC140020FF0B063045
:101B400010B5064C2368186804F0C6FA2020FEF78A
:101B5000D9FE2368043B236010BDC046EC1400206E
:101B6000F0B587B003AA2A4B13CB13C2294B1A68CE
:101B700001929A8801AB9A805B20FEF7C3FE264B48
:101B80001B68264A0C3293420DD0244A0C329342F1
:101B90000DD3224A0C32934216D9204C103404251E
:101BA0001E4F160024E001A804F0C5F80CE003A8BD
:101BB00004F0C1F8194B00221A605A609A601800AC
:101BC0000C3015490860DA605D20FEF79BFE20208E
:101BD000FEF798FE07B0F0BD206804F07DFA2020E3
:101BE000FEF790FE01350C4B1B680434B342EBD971
:101BF000DB1B9B10AB42E7D32020FEF783FE084B94
:101C00001B68102BE8D02068FEF756FFE7E7C046B8
:101C1000085D0008145D0008EC1400208813002003
:041C2000C8140020C4
:101C2400F0B5D6464F464646C0B584B001AA394BF6
:101C340003CB03C21B7813702020FEF761FE364BE2
:101C44001B68002B5BD0354D00270026C0231B05E5
:101C54009946334B9A46304B984616E02020FEF7BF
:101C64004FFE14E06B684A46134221D12020FEF750
:101C740047FE2020FEF744FE01360137052F34D8F5
:101C8400103543461B68B34237D9092EE6D93000D4
:101C9400FEF710FF3A20FEF733FE2C00083C2078B4
:101CA4000028DFD0FEF72CFE0134AC42F7D1D9E78F
:101CB40001A804F03EF853461B68102B11D0286885
:101CC400FEF7F8FE2020FEF71BFE4020FEF718FE6C
:101CD4002804000C04F0FEF92920FEF711FE023757
:101CE400C4E7286804F0F6F9ECE70D20FEF708FED7
:101CF4002020FEF705FE0027C2E7002F05D104B01F
:101D0400E0BCBA46B146A846F0BD0D20FEF7F8FD8A
:101D1400F5E7C046E05E0008081500200C08002026
:041D2400C8140020BF
:101D280010B5044C2368186804F0A7F82368043B2E
:081D3800236010BDEC14002033
:101D4000F0B5C64600B582B06846214B020012CB02
:101D500012C203F0F0FF0D20FEF7D4FD1D4DFA2353
:101D60009B009846A8440026012723E0FEF7CAFD01
:101D70000134285D0028F9D1062C05D82020FEF773
:101D8000C1FD0134072CF9D12320FEF7BBFD38003B
:101D900003F0FBFF2020FEF7B5FD2020FEF7B2FD8B
:101DA0002020FEF7AFFD01370136052E07D008359C
:101DB000A84509D02020FEF7A5FD0024D9E70D2075
:101DC000FEF7A0FD0026F2E702B080BCB846F0BDE9
:081DD000C85400080058000887
:101DD80070B5A8B0DB4B1A6826929A8869469C2091
:101DE80009180A809B796A469E215218137023AC01
:101DF800D54B220023CB23C221AAD44B19682191A9
:101E0800998891809B7993711FAAD14B03CB03C208
:101E18001CAAD04B03CB03C211001A880A809B78F6
:101E28008B7019AACC4B23CB23C215AACB4B23CB3F
:101E380023C21B78137012AAC94B03CB03C21B8899
:101E480013800FAAC74B03CB03C21B8813800DAAAC
:101E5800C54B03CB03C20AAAC44B03CB03C21B78EE
:101E68001370C34B099307AAC24B03CB03C2C24BDF
:101E78001A6805929A8805AB9A8002AABF4B03CBD1
:101E880003C21B7813706A46BD4B03CB03C24420C0
:101E9800FEF734FD6120FEF731FD7420FEF72EFDBC
:101EA8006120FEF72BFD26A803F041FFB5480C3052
:101EB80004F0B2F85220FEF721FD6520FEF71EFD62
:101EC8007420FEF71BFD26A803F031FFAE4804F08E
:101ED800A3F8200003F02BFFAC4804F09DF8552030
:101EE800FEF70CFD7320FEF709FD6520FEF706FDE1
:101EF8007220FEF703FD3D20FEF700FDA44804F024
:101F08008BF80D20FEF7FAFCA24B1B68002B00D1C2
:101F1800D9E01FA803F00BFF9E4B1B68002B00D0D5
:101F2800D5E01CA803F003FF9B4B1B680024002B83
:101F380000D1D6E0964E984D2B68013B1B01F31853
:101F4800185D002804D0FEF7D9FC0134082CF3D121
:101F580019A803F0ECFE914B186830231843C0B25F
:101F6800FEF7CCFC15A803F0E2FE8D4D8D4E3268CD
:101F78005101891A8B01591AC900891889012868E1
:101F880004F0D0F80400FEF793FD2E20FEF7B6FC0F
:101F980033685A01D21A9100C918C900286804F098
:101FA800C1F863011B1B9B001B19DB00C01AFEF75D
:101FB8007FFD4D20FEF7A2FC4820FEF79FFC7A200B
:101FC800FEF79CFC0D20FEF799FC12A803F0AFFE6B
:101FD800754C2068FEF76CFD23680B2B00D18DE053
:101FE800714B1B68132B00D18FE06F4B1B68262B9E
:101FF80000D18EE06C4B1B68392B00D18DE030206E
:10200800FEF77CFC3020FEF779FC684B1B68002B40
:1020180000D186E02020FEF771FC2020FEF76EFC40
:102028005320FEF76BFC5020FEF768FC4920FEF7B2
:1020380065FC3D20FEF762FC5D4B1868FEF738FD35
:102048002C20FEF75BFC5B4B1B68102B00D16CE06F
:10205800594B1868FEF72CFD2C20FEF74FFC574B08
:102068001868FEF725FD0DA803F061FE544B1B68A8
:10207800002B00D0A8E00020FEF71AFD0AA803F004
:1020880056FE504B1868002800DADBE0494B1B6805
:10209800102B00D1DAE0FEF70BFD07A803F047FE8E
:1020A8003B4B9B6C013300D0D7E09023DB059B8A28
:1020B800DB0700D5CDE0684603F039FE0D20FEF7BA
:1020C8001DFC28B070BD21A803F031FE21E72320B4
:1020D800FEF714FC2F4B18683030C0B2FEF70EFC28
:1020E8001FE76E20FEF70AFC6F20FEF707FC6E2044
:1020F800FEF704FC6520FEF701FC29E73520FEF712
:10210800FDFB3220FEF7FAFB6AE73220FEF7F6FB0A
:102118006BE73420FEF7F2FB6CE73620FEF7EEFBA8
:102128006DE70FA803F003FE74E7234B186803F06C
:10213800CFFF2C20FEF7E2FB204B186803F0C8FF06
:1021480091E7C046D0540008D8540008E454000869
:10215800EC540008F4540008005500080C55000819
:102168001C55000828550008345500083C5500083F
:102178004F46460048550008505500085855000875
:10218800645500088813002018130020040200205A
:10219800040800205C150020481500206015002068
:1021A80000020020E4140020701500206C150020A7
:1021B800D8140020C8140020E0140020DC140020EB
:1021C8001C150020001500202B4B1E686425754344
:1021D80029002A4803F0A6FF0400FEF769FC6643BD
:1021E800B3059B1B9C01A4196400A419E400244BAB
:1021F8009C4664442E20FEF781FB2900200003F052
:1022080091FFFEF755FC2900200003F0F0FE8C003A
:10221800641864002900200003F084FF06002900E8
:10222800200003F0E4FE880040184000290003F075
:1022380079FF042383429B415B42F6183000FEF786
:1022480037FC1BE709A803F072FD26E703F040FFFF
:1022580023E72D20FEF752FB2DE705A803F067FDC5
:10226800084B1868FEF724FC02A803F060FD064B33
:10227800986CFEF71DFC21E738150020C0C62D001C
:0C22880080C3C901D0140020040800200D
:1022940010B588B001A91F4B0A0013CB13C213CB8E
:1022A40013C21B6813601C4A13681C68043B136048
:1022B400112C17D0192C28D0382C0FD12624132CEC
:1022C40014D0262C12D0392C10D0602C0ED0134AE6
:1022D4008023DB0011680B43136014E0572C02D1F8
:1022E400392403E00B24962C10D1602401A803F0B8
:1022F40020FD0D20FEF704FB094B1C60FDF7C4FF15
:10230400084B00221A6008B010BD13240B2CEDD02A
:10231400D5E7C0466C550008EC14002024150020B5
:08232400701500206C1500206B
:10232C0070B5FEF74DFD041E00D1D7E0C0B26F4B67
:10233C001B68002B08D06E4B1B68002B04D06D4B18
:10234C0018706D4B01221A600A2800D1C3E00228D4
:10235C0000D8C2E0664B1C68002C08D109281ED09E
:10236C00664B1B683F2B02D9202800D19DE0282802
:10237C0017D02F283FD01B2867D1002C00D1ADE0FF
:10238C000E38FEF7B9FA5D4B1A685D4B2021995453
:10239C009B18002159705B4B1A6002249EE0173089
:1023AC00DEE7594B1C68002C01D0002496E0FEF7A8
:1023BC00A3FAFEF705FD0028FBD0C0B220280BD0F5
:1023CC004E490B684E4A2825D554D218507002330A
:1023DC000B60FEF791FA81E0484B1B6801334A4AC7
:1023EC0013601838FEF788FA2020FEF785FA0820CB
:1023FC00FEF782FA72E0444B1C68002C01D00024DA
:10240C006CE0FEF779FAFEF7DBFC0028FBD0C0B2DB
:10241C002F280BD039490B68394A2F25D554D2189F
:10242C00507002330B60FEF767FA57E0334B1B68B2
:10243C000133354A13602738FEF75EFA2020FEF789
:10244C005BFA0820FEF758FA48E0092848D0122811
:10245C0048D0082817D12C4B1D680024002D3DD1E5
:10246C00264B1C68002C39D0013C1C60244B2022CC
:10247C001A55FEF741FA2020FEF73EFA0820FEF727
:10248C003BFA2C002AE00D2817D11C4B1B68002BA3
:10249C000BD11A4B1A681A4B202199549B18002106
:1024AC005970184B1A60012418E0174B1B68012B4C
:1024BC00EFD00D20FEF720FAEBE7134B1C68002C35
:1024CC0012D10E4D0E4B2A689854FEF715FA2B6854
:1024DC0001332B6002E0002400E00024200070BDDA
:1024EC000324FBE70424F9E70024F7E7F8010020B4
:1024FC002015002074150020C4140020B8140020EE
:0C250C00F8130020BC1400202C15002047
:1025180010B5154B1968154B5A5C202A09D14B1C6C
:102528001248013819000133C25C202AFAD00E4B38
:1025380019600023002A10D00C4840180C4CC25CCB
:10254800202A03D01A5501330F2BF8D1084A00204E
:10255800D0545B18074A136010BD054B00221A704F
:10256800044B1960F8E7C046AC140020F8130020AB
:082578005C140020B8140020DF
:10258000F0B5DE46474680B587B00E0002AA0024AB
:1025900005E0002B1BD001340132102C08D0035D64
:1025A0001370190061391929F3D8203B1370F2E731
:1025B000002302AAD37313782D2B0ED1254B0022B2
:1025C0001A6001239B460127012C0FD82CE0002321
:1025D00002AAD37313782D2B2CD01E4B00221A6025
:1025E00000239B4600270120002C2DD0194B1D688D
:1025F000B84602AB9C46E04400230193434618785A
:10260000310003F052FC431C18D075432D180137DC
:1026100001239C46E0440193A742EFD30D4B1D607C
:1026200001205B46002B0FD00A4A13685B421360FF
:10263000012009E00020012CC0D105E0019B002B06
:1026400001D0044B1D60002007B0C0BCBB46B046A3
:08265000F0BDC046B0140020EB
:1026580010B5344B187800285AD00023314901337B
:102668005A5C002AFBD12D280FD0302829D12D4AB9
:10267800527820218A43582A11D02B4A11681029F0
:102688003AD1082B48D900204BE0012B3AD0264AF2
:10269800116810292AD00B2B3ED9002041E0214A8D
:1026A80092782D2A09D00A2B2ED81E4810210230E4
:1026B800FFF762FF431E984133E00B2BF5D900204A
:1026C8002FE02528D9D1174A52782D2A09D00B2B6B
:1026D8001CD814480A210130FFF74EFF431E9841C9
:1026E8001FE00C2BF5D900201BE000232D28C8D1B2
:1026F800092B11D9002014E02D28CCD000200A2B5A
:102708000FD809E000200CE000200AE0002008E0D3
:10271800054B19681029E8D00248FFF72DFF431E22
:0C272800984110BD5C140020C814002073
:10273400F0B51A4C00251A4E0021635C8A5D18001E
:10274400613819280DD8203BDBB2100061381928F4
:1027540011D8203AD2B2934219D101310829ECD1CF
:1027640015E01000613819280DD918002038471ECB
:10277400B84140420340934209D1002AEDD1094BAC
:102784001D600120F0BD203AD2B2202BE3D10135E7
:1027940008347E2DD0D10020F4E7C046F857000855
:0827A4005C140020FC1400206D
:1027AC0070B51A4B1B78002B29D0194A00231E0038
:1027BC00013310321100103909780029F7D1731C3C
:1027CC001FD03301114C1C19124D16E08B4211D144
:1027DC0000290BD00132082A0CD0A15C535D1800E3
:1027EC0061381928F2D8203BDBB2EFE70A4B1E60A8
:1027FC00012070BD103C013E05D30022EDE7002006
:10280C00F7E70020F5E70020F3E7C04604080020B6
:0C281C00140800205C140020FC140020B4
:1028280010B50F4B1A680F4B1A60FFF771FEFFF7D0
:10283800B9FF002805D00C4B1B6801330B4A136005
:1028480010BD0B4B1B78302B05D00A4A2123116889
:102858000B431360F4E7054B00221A60F0E7C0460B
:10286800B8140020AC140020FC14002048150020E7
:082878005C140020241500206F
:10288000074A13680749C85401331360064A934244
:1028900004D9064A202311680B4313607047C046D1
:1028A0003415002004020020FE050000241500203D
:1028B00010B5144B18688200134BD3581A030AD46E
:1028C000124A1268002A13D19B030BD48000104BCC
:1028D000C358984705E00F4A80239B0011680B43BB
:1028E000136010BD0B4A082311680B431360F8E70F
:1028F000DB0304D58000064BC3589847F1E7FFF788
:10290000BFFFEEE7FC140020005600082815002049
:08291000000000202415002046
:1029180070B594B00CA9414B0A0013CB13C213CB6A
:1029280013C203CB03C205A93D4B0A0013CB13C244
:1029380013CB13C21B7813706A463A4B13CB13C2DE
:1029480011001A680A601B790B71374B1B68522BF0
:1029580009D95224354E344DA05DFDF7CFFF01341F
:102968002B68A342F8D85223314A1360314A002118
:102978001160314A13602E4D304E03E02C4B1A681B
:102988002D4B1A60284C2B682268934234D2FFF7EB
:10299800BFFD3378002BF6D0FFF75AFE00280BD086
:1029A800274B1A68274B1A60274B1B68002BE5D06A
:1029B800264B01221A60E1E7FFF7B8FE002811D084
:1029C800234B1B689B00234A9B585B0321D5FFF7C9
:1029D8006BFF214B1B68002B08D1154B1A68164B4F
:1029E8001A60CFE70CA803F0A2F905E01A4B002201
:1029F8001A60684603F09BF90D20FDF77FFF52230C
:102A0800094A13600A4A13600A4B00221A6014B07C
:102A180070BD05A803F08BF9EEE7C046F85E000824
:102A2800185F0008345F0008BC140020F813002069
:102A3800B81400202C150020AC1400205C140020D1
:102A4800B01400203C15002020150020401500205F
:0C2A5800FC14002000560008241500208B
:102A640070B56E20FFF70AFF0C4D2C68FF20FFF7AE
:102A740005FFFF20FFF702FF2B68013B084A9B1864
:102A84001B04180C074909681B0E0D6853550B6885
:102A94009C46624450700C6070BDC04634150020E2
:082AA40004020020EC140020E4
:102AAC0010B56F20FFF7E6FE064A1368191D11607A
:102ABC00054A12685A60FF20FFF7DCFEFF20FFF783
:0C2ACC00D9FE10BDEC14002034150020D1
:102AD80010B57320FFF7D0FE064A1368191D116060
:102AE800054A12685A60FF20FFF7C6FEFF20FFF76D
:0C2AF800C3FE10BDEC14002034150020BB
:102B0400F8B57420FFF7BAFE104E33681D6801351E
:102B14000F4C2D19280AFF273840FFF7AFFE380065
:102B24002840FFF7ABFE0B4B1B68013B1B193268B7
:102B3400190A106821541268A41863707620FFF7EC
:102B44009DFE3368043B3360F8BDC046EC1400209E
:082B54000402002034150020EA
:102B5C0010B5234B1B68002B17D1224B1B68224A44
:102B6C0019681160214A93422ED9214A1268022A0F
:102B7C001DD0043B1B4A13601E4A1368013B1360B3
:102B8C001D4B1A681D4B1A6010BD6420FFF772FEB6
:102B9C000022134B1A601A490B6801330B601B019E
:102BAC0018495A54184B1A68184B1A60E8E7114A1E
:102BBC001168174A12689142DBD1154A0021116045
:102BCC000B4A03311160D4E7074B00221A60084B03
:102BDC001B68022BD4D1064B03321A60D0E7C046D7
:102BEC0028150020F41400201815002018130020BC
:102BFC00F80100200C15002004150020C81400203A
:102C0C000815002004080020341500203015002081
:042C1C00441500203B
:102C200070B5324B1B68002B27D1314B1B681C78C9
:102C300023005F3B022B16D97D20FDF763FE202089
:102C4000FDF760FEFEF78CFF25006F3D072D15D9BF
:102C5000733C012C1CD9032D0FD8264B1B681888F8
:102C600003F004FA09E0244B186801300005000D58
:102C700003F0FCF92920FDF745FE70BD2020FDF78B
:102C800041FE5220FDF73EFE3A20FDF73BFEDFE716
:102C9000184B1A68194BD31A082BEED90C3A108826
:102CA00003F0E4F92020FDF72DFE2020FDF72AFE99
:102CB000104C2368083B188803F0D8F92020FDF752
:102CC00021FE6920FDF71EFE2368043B188803F0EF
:102CD000CDF92020FDF716FE7820FDF713FE2368BE
:102CE0001888013003F0C2F9C7E7C0462415002058
:102CF00014150020F41400201815002018130020CB
:102D0000084B1868084B1B68984208D001D2181A63
:102D10007047C01A80239B009C466044F8E700205F
:0C2D2000F6E7C0464C15002050150020BE
:102D2C0010B5094B1C68221D1A60084B1B68002B40
:102D3C0006D0074B1B68002B02D0064B186801E02D
:102D4C00FFF7D8FF606010BDEC140020F8010020E4
:082D5C0020150020C414002022
:102D640010B50B4B1C6800230A4909190A48CA5CB0
:102D7400222A03D01A5401334F2BF8D1064A2221B8
:102D8400D15401330021D154E318044A136010BD17
:102D9400AC140020F81300205C140020B8140020A8
:102DA4001A4B1B185A781300613B192B03D8203A8D
:102DB4001300373B05E02F2A1BD91300303B092BA6
:102DC400F6D80F2B18D8114A1018827811006139DF
:102DD400192907D8203A373A11000F2912D81801B7
:102DE400401870472F2A0AD9110030390929F4D91B
:102DF400F1E701204042F4E701204042F1E70120DD
:102E04004042EEE701204042EBE7C0465C1400205C
:102E140070B5324B1B680133314A1360FFF7A0FFD2
:102E2400002600242F4A03E001360134502C0ED032
:102E3400A35C5C2BF8D0222BF7D12A4B00221A5525
:102E4400294B1D68002D08D1264C260032E0274A64
:102E5400022311680B4313603EE06520FFF70EFD6B
:102E6400234A13687600A41B2249CC54013313600F
:102E740000241C4D2E0005E0FFF700FD0134335DF6
:102E8400002B29D0285D5C28F6D12000FFF788FFAD
:102E9400431C03D00334FFF7F1FCF0E7134A022389
:102EA40011680B43136017E0FDF72AFD0135735DCC
:102EB400002B11D0605D5C28F6D12800FFF770FF6D
:102EC400431C04D00335C0B2FDF71AFDEFE7074AEF
:102ED400022311680B43136070BDC046B814002070
:102EE400AC1400205C1400202815002024150020B8
:082EF400341500200402002047
:102EFC0070B52F4B1C6824012E4B1D682900200037
:102F0C0003F00EF92C4B186080235B02984227D3F8
:102F1C00294B2A4A1A602A4B1B88DB0710D4284BF2
:102F2C0000221A821A802749CA6902200243CA6108
:102F3C00254A1A836422DA621A8801210A431A800C
:102F4C001D4B1B68013B9BB21D4A13851F4B1B6815
:102F5C00002B27DB1A4A138C01210B43138420E02E
:102F6C00AC42D8D2164A13880124A3431380002301
:102F7C0017490B6017490B60144B0121494219602A
:102F8C009023DB051868144D28401860D968294037
:102F9C00D960D868802189010143D960138CA3437F
:102FAC00138470BD138C01218B431384F9E7C04645
:102FBC0038150020E41400201C150020FFFF000031
:102FCC00000400400010024060600000001500206A
:0C2FDC00B4140020F8140020FFCFFFFF09
:102FE8009022D205136827490B401360264A138C98
:102FF80001218B431384254B1B68002B22DB902176
:10300800C905CA681F480240CA60002B22D0632B3A
:103018002ADC9023DB051968802292010A431A6092
:103028001A6A1B490A401A62196A802252040A4322
:103038001A62154B1A8C01210A431A84134A126822
:103048005A6370479022D205D16880239B010B43B5
:10305800D360F6E70B000968802252010A431A6020
:103068008022D2039A61ECE7084B64221A6090230D
:10307800DB051968802252010A431A6040229A61CE
:10308800DFE7C046FFCFFFFF000400400015002027
:04309800FFFFFFF047
:10309C00324B9B6C002B60DD314A1268002A29DB15
:1030AC0030490A60304A1268022A1ED008DC002A15
:1030BC000ED0012A45D19022D205022191610FE058
:1030CC00032A3ED19022D2058021890291613EE0F3
:1030DC009022D2058021490291618021890291615F
:1030EC0021490A6801320A6034E09022D20501219C
:1030FC009161F5E752421B490A601B4A1268022A89
:10310C001AD008DC002A0ED0012A1AD19022D2053E
:10311C0001219161E4E7032A13D19022D205802189
:10312C004902916113E09022D205802149029161FC
:10313C00802189029161D3E79022D205022191610D
:10314C00CEE709490A6801320A60032A02DD064A01
:10315C0000211160013B014A936470470408002070
:0C316C00D0140020E8140020D41400202F
:1031780070B500230D4A13600D4A13600D4A1360A1
:103188000D4C0E4D0E4E03E0FFF7CCF800280BD186
:10319800A36C002BF8D02B68002BF5DD3368002BCF
:1031A800F2D1FFF777FFEFE7012070BDB8140020D8
:1031B800BC1400202C15002004080020D014002086
:0431C800E8140020E7
:1031CC0070B522490B681A6821480260043B0B60F9
:1031DC00002A39D01F4C204D204E0FE0204B1B688D
:1031EC00022B19D01F4B1B68002B03D01E4B1B68E6
:1031FC00002B15D1164B1B68002B25D0FCF7C8FFF4
:10320C00A36C002BEAD02B68002BE7DD3368002B76
:10321C00E4D1FFF73DFFE1E7114B00221A6013E008
:10322C00FFF77EF8012806D0022807D00F4B1B6849
:10323C00002BDFD008E0FFF769FBF7E70B4A802390
:10324C005B0011680B43136070BDC046EC1400208A
:10325C001015002004080020D0140020E8140020D1
:10326C00C0140020F8010020201500202415002097
:10327C0010B5044B1A68642311684B431360FFF7B5
:08328C009FFF10BDEC140020AF
:10329400074A13681868043B1360112806D0F0230A
:1032A4000340A02B01D1913B18407047B120FCE7AB
:0432B400EC140020F6
:1032B80070B5FFF7EBFF254B1B68002B20D10F28BB
:1032C8002ED80300083B042B1BD90F2819D0204BFC
:1032D8001B68013301D0062818D044000322A240FD
:1032E8009023DB05D9689143D96019689143196027
:1032F8001D6801221100A1402943196082409A618A
:1033080070BD124B8022D2001A60F9E7114A138C63
:1033180001218B4313840E4B012252421A60DCE7D1
:10332800B12804D0094B8022D2001A60E8E70A4B82
:10333800DA680C218A43DA601A688A431A601A68C4
:1033480008390A431A6002229A61D9E72415002035
:0C335800001500200004004000040048A4
:1033640070B5FFF795FF264B1B68002B21D10F2862
:103374002FD80300083B042B1CD90F281AD0214B4B
:103384001B68013301D0062819D044000322A2404F
:103394009023DB05D9689143D9601968914319607A
:1033A4001D6801221100A140294319601030824098
:1033B4009A6170BD124B8022D2001A60F9E7124A5A
:1033C400138C01218B4313840E4B012252421A6049
:1033D400DBE7B12804D00A4B8022D2001A60E8E768
:1033E4000A4BDA680C218A43DA601A688A431A6045
:1033F4001A6808390A431A60802292029A61D8E74F
:10340400241500200015002000040040000400489A
:1034140010B5FFF73DFF234B1B68002B1DD10F2870
:103424002BD80300083B042B18D90F2816D01E4BA9
:103434001B68013301D0062815D0400003228240C6
:103444009023DB05196891431960D9689143D960C9
:10345400D968012282400A43DA6010BD114B8022F0
:10346400D2001A60F9E7114A138C01218B431384AB
:103474000D4B012252421A60DFE7B12804D0094BF8
:103484008022D2001A60E8E7094B1A680C218A43AB
:103494001A60DA688A43DA60DA6808390A43DA605B
:1034A400DBE7C0462415002000150020000400407E
:0434B40000040048C8
:1034B80010B5FFF7EBFE234B1B68002B1DD10F281F
:1034C8002BD80300083B042B18D90F2816D01E4B05
:1034D8001B68013301D0062815D040000322824022
:1034E8009023DB05196891431960D9689143D96025
:1034F800D968022282400A43DA6010BD114B80224B
:10350800D2001A60F9E7114A138C01218B43138406
:103518000D4B012252421A60DFE7B12804D0094B53
:103528008022D2001A60E8E7094B1A680C218A4306
:103538001A60DA688A43DA60DA6804390A43DA60BA
:10354800DBE7C046241500200015002000040040D9
:043558000004004823
:10355C0010B5FFF799FE1E4B1B68002B18D10F28D6
:10356C0026D80300083B042B13D90F2811D0194B74
:10357C001B68013301D0062810D040000322824082
:10358C009023DB05196891431960D9689143D96080
:10359C0010BD0F4B8022D2001A60F9E70E4A138C33
:1035AC0001218B4313840B4B012252421A60E4E736
:1035BC00B12804D0064B8022D2001A60E8E7074BF2
:1035CC001A680C218A431A60DA688A43DA60DFE7EA
:1035DC0024150020001500200004004000040048C1
:1035EC0010B5FFF751FE104B1B68002B0FD10F28A5
:1035FC000ED89023DB051B8A0122824013400B4915
:10360C000A68101D0860002B0AD00123536010BDFE
:10361C00074B1B8A0F2210400E3A82401340EEE7F4
:10362C0000235360F3E7C04624150020EC1400205F
:04363C00000400483E
:1036400010B5144BDA6814490A40DA60996980228F
:1036500092000A439A6102F052FB02F050FB02F022
:103660004EFB02F04CFB0D4B0022DA608021090674
:103670001961022159610A490A609A6801210A43C5
:103680009A60190001220B681A42FCD002F037FB45
:1036900010BDC04600100240FFFDFFFF00240140A6
:0436A00008270140B6
:1036A4000C4B1A6801210A431A609A6801310A43D3
:1036B4009A60190001228B681A42FCD1064B9A6960
:1036C40006490A409A61D968802292000A43DA6066
:1036D4007047C0460024014000100240FFFDFFFF78
:1036E400F0B5C64600B52C4B802252049A61FFF710
:1036F400D7FF2A4BDA6801218A43DA609A690A43C0
:103704009A619024E4052668E26890462268C02005
:1037140082432260E2688243E260E26880380243C6
:10372400E2601F480022826002611E480260812715
:10373400FF004760C7601C48076904252F430761E1
:103744005D698027FF032F435F61184F3A60184D6E
:10375400FD60BFF34F8FBFF36F8F40BF20BF20BF0B
:1037640002615A69134802405A61DA680A43DA600E
:1037740002F0C3FAFCF7A2FC0F4B104A1360104A84
:10378400136026604346E36002F0B7FA5E20FDF75B
:10379400B7F880BCB846F0BD0004004800100240F1
:1037A400000001400004014000ED00E00014004866
:1037B400AAAAAAAAFFFFBFFF1411002050150020D7
:0437C4004C15002080
:1037C800F0B589B004AA5C4B13CB13C21B881380D5
:1037D8006A465A4B13CB13C21B781370584B1B689D
:1037E8001C68621C18D0072C03D92300A03B072BA8
:1037F8001BD8544B9B699B051ED5534B534A1A60E3
:103808000F232340590003228A40072B00D990E058
:1038180099004F4841588F46043B494A1360FFF7C7
:103828003DFF684602F083FA35E04A4A8023DB0010
:1038380011680B4313602EE0FFF7FEFE04A802F0A8
:1038480076FADAE79021C905086810430860C86865
:103858009043C86001229A4013003B4A93620426B1
:10386800002714000425A3682B43A36023681D4286
:10387800FCD0236CFF1802F03EFA013E002EF2D174
:103888002F4B1B68BA081A60BB0704D52C4B1A6863
:1038980013680133136009B0F0BD9021C9050868A9
:1038A80010430860C8689043C860D3E79021C905F1
:1038B800086810430860C8689043C860CAE7902148
:1038C800C905086810430860C8689043C860C1E724
:1038D8009021C905086810430860C8689043C8600B
:1038E800B8E79021C905086810430860C868904384
:1038F800C860AFE718490968013108D01748018C3A
:103908000124A14301841449012040420860902108
:10391800C905086810430860C8689043C86099E7FB
:103928009021C905086810430860C8689043C860BA
:1039380090E700238EE7C046545F0008645F0008E4
:10394800EC1400200010024000240140FF07000092
:1039580088550008241500200015002000040040A8
:103968001B4B1B68032B26D81A4B1B68043B1C2BCC
:1039780021D880235B02184A12689A421BD29023EE
:10398800DB051A6815490A401A6019688222520034
:103998000A431A60DA6803218A43DA60DA6801396F
:1039A8000A43DA600A4B1B68012B0BD99023DB050D
:1039B80002229A6105E00A4A8023DB0011680B4362
:1039C800136070479023DB05802292029A61F8E722
:1039D800D8140020E0140020DC140020F0FCFFFFC5
:0439E8002415002082
:1039EC0010B50A4A13680A4918680860191F116053
:1039FC000868084908601900083911600868064908
:103A0C0008600C3B1360FFF7A9FF10BDEC140020FD
:0C3A1C00DC140020E0140020D81400206E
:103A2800F0B5DE4657464E464546E0B583B090238E
:103A3800DB051B68434A13408222520093421FD180
:103A4800414B1C68012C1ED99023DB0502229A6188
:103A58003E4B1B689B461B6801933D4B19683D4BC9
:103A68001D68002201269020C00580235B039A462A
:103A78001023994680239B02984602239C4637E0F0
:103A8800FFF76EFFDCE79023DB05802292029A6144
:103A9800DEE75346836133E0012C0CD99023DB0524
:103AA800023199615B461A6003B0F0BCBB46B2466E
:103AB800A946A046F0BD9023DB05802189029961C3
:103AC800F0E743468361002D2CD15200038A33402E
:103AD8001A4303E05200038A33401A436346836162
:103AE8002B00002B02D0013B002BFCD10029D3D0A6
:103AF800013933008B40019F1F42CAD04B46836176
:103B0800002C0BD0032CDCD063468361002D09D137
:103B18005200038A33401A432B0010E04346836166
:103B2800002DD7D02B00013B002BFCD15200038A7B
:103B380033401A43002CD1D02B00032CCED047465B
:103B48008761CEE70F030000D8140020EC14002092
:083B5800E0140020DC14002041
:103B600010B5074A1368191D1160064A12685A6099
:103B7000FF20FEF785FEFF20FEF782FE10BDC04647
:083B8000EC14002034150020B4
:103B8800F8B5104E33681D6801350F4C2D19280AF9
:103B9800FF273840FEF770FE38002840FEF76CFE1D
:103BA8000A4B1B68013B1B193268190A106821541B
:103BB8001268A41863707520FEF75EFE3368043B34
:103BC8003360F8BDEC1400200402002034150020F6
:103BD80070B57D280DD8C0000E4D441908352D1834
:103BE8002078002804D0FCF789FE0134AC42F7D1D4
:103BF80070BD7F2528400001074D441908352D1850
:103C080020780028F4D0FCF779FE0134AC42F7D1D3
:0C3C1800EEE7C046F85700080408002042
:103C240070B50001064D441908352D182078002878
:103C340004D0FCF765FE0134AC42F7D170BDC04638
:043C44000408002050
:103C4800F0B5C64600B582B0AA4B1A6800929B88A8
:103C58006A469380A84B1D68002D03D002B080BC33
:103C6800B846F0BDA54B1B68A54A13601B7898465B
:103C78001F00A44B1B685E00F6180D20FCF73EFEE3
:103C8800002E06D02C002020FCF738FE0134A64276
:103C9800F9D19B4B188802F0E5F92020FCF72EFE9D
:103CA800404602F0DFF92020FCF728FE7E2F1AD8C4
:103CB8004046FFF78DFF6A2F53D06B2F57D06C2FDC
:103CC80000D182E06D2F00D187E06E2F56D0702F83
:103CD80000D18AE0712F00D18DE0FD224346723B6E
:103CE80013424BD059E02D20FCF708FE3E20FCF78C
:103CF80005FE2020FCF702FE4046FFF769FF7F4BD8
:103D08001B685B787F241C40682F00D19EE0692FD8
:103D180000D1A5E0642F00D1C6E07B4C032D00D173
:103D2800D6E02368022B00D8D2E0FCF733FAFEF77E
:103D3800E3FF0028F2D0FEF7F5FA0500012800D1CC
:103D4800BCE0022800D1BCE00428E7D16D4B1B6819
:103D5800002B00D1BCE06D4A13606B4B02221A6045
:103D6800DCE76B4B1B681B68002B07D0C7E7684B69
:103D78001B68191F1A680B689A42C0D0684601F080
:103D8800D6FF5E4B1B68587800029B7818430130B9
:103D980002F068F92920FCF7B1FD662F35D1574BA1
:103DA8001B685C782820FCF7A9FD5A4B1B68102B70
:103DB80027D02000FCF77CFE2920FCF79FFD4F4B05
:103DC8001B685B787F241C40A1E7514B1B681A1FB6
:103DD80012681B689A42D1D291E74D4B1B681A1F93
:103DE80012681B689A42C9D989E7494B1B681B6846
:103DF800002BC3D083E7464B1B681B68002BBDD143
:103E08007DE7200002F064F9D6E7672F00D076E757
:103E18003A4B1A6893781B04517809060B431179B9
:103E28000B43D47824021C432820FCF767FD394B48
:103E38001B68102B06D02000FCF73AFE2920FCF75F
:103E48005DFD67E7200002F043F9F7E72820FCF75B
:103E580055FD2000FFF7E2FE2920FCF74FFD5CE747
:103E68002820FCF74BFD2000FFF7D8FE4020FCF788
:103E780045FD240120000830274E80190004000C5D
:103E880002F026F92320FCF739FD3419A068214BEC
:103E98001B68102B05D0FCF70BFE2920FCF72EFD24
:103EA8003BE702F015F9F8E72020FCF727FD3C2056
:103EB800FCF724FD2D20FCF721FD2EE7FEF728FD59
:103EC8002CE70D4A80235B0011680B431360C5E69D
:103ED8002020FCF713FD43465F3B022B03D86846BE
:103EE80001F025FFBAE67B20FCF708FD2020FCF74F
:103EF80005FDB3E6305D00082415002018150020E4
:103F0800141500200C150020F8010020441500208D
:0C3F1800EC140020C81400200408002055
:103F240010B5FFF78FFE074B1B68002B08D1064B1B
:103F34001B681B789B00054A9B589847FEF76EFE4A
:103F440010BDC046241500201815002000000020D4
:103F540010B51B4A1368013313601A4B1A68111DFC
:103F6400196019490B6853601A787F2313401B01A9
:103F7400164AD3189B680B601B787D2B0BD8144A08
:103F84001268032A04D09B00124A9B58984710BD1C
:103F9400FFF7C6FFFBE70E4B1B68032B06D00E4B47
:103FA4001B68002BF3D1FFF7D3FFF0E7FFF74AFEBE
:103FB400094B1B68002BEAD1FEF730FEEFE7C04641
:103FC4000C150020F414002018150020040800200B
:0C3FD400F801002000000020241500204F
:103FE000F0B587B001AA3F4B13CB13C211001A687A
:103FF0000A601B790B713C4B1B683C4C3C4AA41873
:10400000A34269D23B4D384E2F003EE0FFF7A2FF9E
:1040100045E0FEF775FE00280CD133681B787D2B38
:104020001BD8344A1268032A14D09B00324A9B588A
:10403000984734E0FEF77AF9012808D00228ECD13D
:104040002E4A80235B0011680B43136044E0FEF7A7
:1040500063FCE2E7FFF766FF21E03B68032B02D039
:10406000FFF778FF1BE0FFF7EFFDFEF7D9FDF7E75D
:10407000224B1B68002B2FD11B4B1B68002B1DD024
:104080000133194A1360A34226D22A68002AC0D1FC
:104090001B787D2BBAD89B00174A9B589847184B22
:1040A0009B6C002BE4D0174B1B68002BE0DD164BFC
:1040B0001B68002BDCD1FEF7F1FFD9E70D4B1B6825
:1040C000032B0BD00B4B01221A6000230F4A136005
:1040D0000F4A13600F4A136007B0F0BD01A801F04A
:1040E0002AFEEFE7805F0008181500200402002078
:1040F000F40D0020F801002000000020241500200D
:1041000004080020D0140020E8140020201500200E
:08411000401500200C150020F1
:10411800F8B5274B1C68002C2ED1264B1B681901BB
:10412800254A5218D168C022120511420AD0234AE2
:104138001168081D10601B011F4AD3189B684B604B
:104148002000F8BD1B011C4AD3189A681C4B1A6042
:104158001C4B01221A601C4D2F681C4C26685223E8
:104168002B6023601A4B00221A60FFF735FF2F607F
:104178002660184B1C68E3E70E4B186802010E4BCB
:104188009B18DA68C0231B0514001C401A4204D18E
:1041980080231843FEF770FBD2E76820FEF76CFB1C
:1041A800044B1868FEF768FB0A4B1C68C8E7C04652
:1041B80028150020FC14002004080020EC1400201E
:1041C8001815002020150020BC140020B814002069
:0841D8002C1500202415002025
:1041E00070B50023384A1360384A1360384A1360A8
:1041F0001500384E0EE0384B1B68FF2B24D8662084
:10420000FEF73EFB344B1868FEF73AFB304B1A685A
:104210002E4B1A60314C2B682268934230D2FEF745
:104220007BF93378002BF6D0FEF716FA00281FD062
:104230002B4B1B68002BDED12A4A1368191D116015
:10424000254A12685A60E1E76720FEF719FB224C05
:1042500003202056FEF714FB0223E05EFEF710FB5E
:1042600023681812FEF70CFB2068FEF709FBCDE768
:10427000FEF79CFA002809D0FFF74EFF002800D077
:1042800070BD134B1A68114B1A60C3E7FEF752FA60
:1042900000280AD0FEF70CFB134B1B68002BEFD154
:1042A0000B4B1A68094B1A60B4E70F4A01231168D7
:1042B0000B4313600D4B1A680D4B1A60044B1A68C0
:1042C000024B1A60DCE7C04620150020AC14002029
:1042D000B81400205C140020B0140020BC1400208E
:1042E00028150020EC140020241500203015002093
:0442F0003415002061
:1042F400F0B5DE4657464E464546E0B593B00CA9A8
:10430400BA4B0A0013CB13C203CB03C21B7813703E
:1043140007AAB74B13CB13C211001A680A609A8814
:104324008A809B798B7103AAB24B13CB13C21B886F
:104334001380B14B1A68B14B1A60FEF7EBF8FEF725
:1043440033FA00280DD1FEF7F3F9002805D1AC4A61
:10435400012311680B43136018E10CA801F0E9FC78
:1043640014E1A54B1A68A54B1A6007A801F0E1FCFB
:10437400A44D2B681801A44C001901F0ABFE0D20CC
:10438400FCF7BEFA2B681A01A418E168C0221205D2
:10439400080010400190114200D0FEE01B019A4A2F
:1043A400D3189C68994BE41A2405240D1B5D012540
:1043B400642B00D1D1E0954E24E00D20FCF7A0FA47
:1043C400019D1FE0914B1A195078000202341F5DC1
:1043D40007432820FCF794FA781C01F045FE2920B5
:1043E400FCF78EFA01352020FCF78AFA2020FCF72E
:1043F40087FA0134854B1B5D642B00D1ADE0013598
:10440400072DDAD8A0190004000C01F02DFE3A2083
:10441400FCF776FA305DFFF7DDFB335D1A006A3A8C
:104424000A2ACFD9662B1AD0672B2ED0682B4CD0F2
:10443400692B57D0652BD6D12220FCF761FA734B38
:104444001B195B789B46A31C98465B46002B7DD0CA
:104454006E4B434499465C460F239A466BE0013405
:104464002820FCF74DFA6A4B1B68102B08D0674BC9
:10447400185DFCF71FFB2920FCF742FA0135B2E76F
:10448400624B185D01F026FEF5E760480219937847
:104494001B04517809060B43D7783F020434025DAC
:1044A40013431F432820FCF72BFA594B1B68102B8E
:1044B40007D03800FCF7FEFA2920FCF721FA013571
:1044C40091E7380001F006FEF6E701342820FCF7F6
:1044D40017FA4E4B185DFFF7A3FB2920FCF710FADF
:1044E400013580E701342820FCF70AFA474B1F5DA9
:1044F4003800FFF795FB3F01083743483F18402039
:10450400FCF7FEF93804000C01F0E4FD2920FCF767
:10451400F7F9013567E75C20FCF7F2F9380901F097
:10452400FAFB5046384001F0F6FB013C01239C465F
:10453400E144002C09D04B461F783B00203B5E2B06
:10454400E9D83800FCF7DCF9EFE7D8444446013CED
:104554002220FCF7D5F9033545E72C482018000440
:10456400000C01F081FD3A20FCF7CAF93B20FCF76E
:10457400C7F9244B1A681201234B9B18DA68C0232D
:104584001B051A4209D10D20FCF7BAF913B0F0BC8F
:10459400BB46B246A946A046F0BD03A801F0C9FB3C
:1045A4001B4B1B68102B18D0164B1A681201164BA4
:1045B4009B18986801F063FC2020FCF7A1F94020C7
:1045C400FCF79EF90F4B1868000108300E4BC01819
:1045D4000004000C01F07EFDD5E70A4B1A681201B5
:1045E400094B9B18986801F075FDE5E7505D0008DC
:1045F400685D00087C5D0008B8140020AC1400203D
:1046040024150020FC1400200408002004020020CB
:04461400C8140020A6
:10461800134B1B68134A1360134A1268120113499B
:104628005218BE20C000844661448A420AD210490A
:104638000139891A8908013189005118002001C2FD
:104648008A42FCD10B4A934209D80B4A9B180B4962
:104658008C4662440021197001339342FBD17047A4
:10466800341500203015002008150020040800200B
:10467800F40D0020FE05000004020020FF050000E4
:1046880010B5164B1A68164B1A60FDF741FFFEF776
:1046980089F800280DD0114B1A68114B1A60114B7C
:1046A8001B68042B0BD8104A802311680B43136036
:1046B80004E00D4A212311680B43136010BD0B4A17
:1046C80013600B4A1B0100219954D318DB681B05A2
:1046D8001B0D084A1360FFF79BFFEFE7B814002093
:1046E800AC140020FC14002024150020081500201C
:0846F800040800203415002025
:1047000010B50023204A1360204A1360204A13602A
:10471000204A1360204A1360204A01211160204A78
:104720001360204B1A68204B1A60204A002311782E
:10473000002903D0013310325F2BF8D11C4A1360DB
:104740001C4A1D4BD35C642B1CD01B4B1100013B3E
:10475000CA5C642A02D0002BF9D102E0002B00D001
:104760000133164A1360FFF757FF154A154B1A60BD
:1047700000231360144A0F491160144A1360FCF7B8
:10478000A7FF10BD0C4BEBE72C15002028150020CF
:1047900020150020401500200C150020F8010020F5
:1047A000C414002004150020C814002004080020B0
:1047B0000815002004020020FF0500003415002029
:1047C00018130020F41400201815002024150020D0
:1047D00030B5B3B030AA984B196830919988918060
:1047E0009B7993712EAA954B19682E919988918087
:1047F0009B7993712BAA924B03CB03C211001A88A9
:104800000A809B788B7028AA8E4B13CB13C225AAE3
:104810008D4B03CB03C211001A880A809B788B70E2
:1048200021AA8A4B13CB13C21B8813801BA9884B68
:104830000A0013CB13C203CB03C21B78137017AA51
:10484000844B13CB13C21B68136013AA824B13CB88
:1048500013C21B8813800EAA804B13CB13C2110006
:104860001A680A609B888B8008A97D4B0A0013CBCD
:1048700013C203CB03C21B78137004AA794B13CB6A
:1048800013C21B7813706A46774B13CB13C21B8875
:104890001380764B1A68764B60339A4200D27CE0E4
:1048A00074490423086803430B60714B0C339A422C
:1048B00004D2704A042311680B4313606E4B1B68CB
:1048C000002B0FD06D4B19686D4B09010022CA54A3
:1048D0005B185A709A70DA701A715A719A71DA719B
:1048E0009A60DA60644B00221A60664B1B68002BEA
:1048F0000ED00024634D2020FCF704F801342B680F
:10490000A342F8D85E20FBF7FDFF0D20FBF7FAFF6E
:1049100030A801F010FA574C206801F0A7FB3D20A9
:10492000FBF7F0FF2368DB075AD4524B1B689B0749
:104930005AD4504B1B685B075AD44E4B1B681B075D
:104940005AD44C4B1B689B065AD44A4B1B681B0617
:104950005AD4484B1B68DB055AD4464B1B689B0551
:104960005AD4444B1B685B055AD4424B1B681B0549
:104970005AD42EA801F0DFF9424B1868FCF79CF8D6
:104980002920FBF7BFFFFFF7BBFE0D20FBF7BAFFA7
:104990003D4B00221A6033B030BD354B0C339A4288
:1049A00000D286E7334B1B68002B00D086E7324BE2
:1049B0001B68002B3CD1354B1B68012BE5D0202018
:1049C000FBF7A0FF6F20FBF79DFF6B20FBF79AFF23
:1049D0002F4B1B68102BD8D14820FBF793FFD4E74F
:1049E0002BA801F0A8F9A0E728A801F0A4F9A0E7F6
:1049F00025A801F0A0F9A0E721A801F09CF9A0E703
:104A00001BA801F098F9A0E717A801F094F9A0E716
:104A10000EA801F090F9A0E713A801F08CF9A0E727
:104A200008A801F088F9A0E704A801F084F9A0E73C
:104A3000684601F080F9A8E7BC5D0008C45D000885
:104A4000CC5D0008D85D0008E45D0008F05D00085A
:104A5000005E0008185E0008285E0008385E000846
:104A60004C5E0008645E0008745E0008EC140020D0
:104A70008813002024150020281500200815002088
:104A800004080020AC140020401500202C15002044
:044A9000C814002026
:104A940010B50023274A1360012227490A602749D9
:104AA4000B6027490A60274A5168F020814351600E
:104AB40051685160244A1360244A08211160244A31
:104AC4002A311160234A1360234A1360234B0122C5
:104AD40052421A60224B323256240021C020000573
:104AE4001C705A709970D860996010330132D2B238
:104AF400352AF5D11A4B0B324E2199540132053126
:104B040099540132013199540439013299540022E3
:104B140044201A54C0200005D864012040429864FF
:104B24001048052404605A540F4B1A60FFF7E6FD41
:104B340010BDC0465C150020F80100204815002077
:104B4400E414002000100240D8140020E0140020D7
:104B5400DC140020381500201C150020001500204E
:0C4B640004080020081500203415002073
:104B700070B5164C164D2B682360FDF7CDFC2B68E5
:104B80002360144B1D68013D28006B1C17D02D01BC
:104B9000114BED18114E10E08B420BD1002913D0B0
:104BA0000132A95C935D1C00613C192CF4D8203BB8
:104BB000DBB2F1E7103D013804D30022F1E7012018
:104BC000404201E00120404270BDC046AC140020CC
:104BD000B814002008150020040800205C140020F0
:104BE00010B5FFF7C5FF0400431C0DD002011D4B9B
:104BF0009B18DA68C0231B051A420BD01A4A80237F
:104C000011680B43136010BD174A212311680B4331
:104C10001360F8E7FFF7ACFF431C11D00201114B02
:104C20009B18DA68C0231B051A420FD1844213D99E
:104C30000C4B24011C19A268000118188260E2E7DD
:104C4000094A212311680B431360DCE7064A8023DD
:104C500011680B431360D6E7034A802311680B43A6
:0C4C60001360D0E7040800202415002099
:104C6C0010B5FFF77FFF431C0FD003010D4AD2187C
:104C7C00D3681B051B0D0C495B1892689A420AD32A
:104C8C000001084A1018836010BD084A21231168DE
:104C9C000B431360F8E7054A802311680B4313603C
:104CAC00F2E7C0460408002004020020241500206E
:104CBC00074B1A68511C196051780902901C186036
:104CCC0092781143802292050A431A607047C046BD
:044CDC001815002087
:104CE00010B5084B1B681B68002B08D0064A1368D8
:104CF00002331360034A1368043B136010BDFFF7CF
:0C4D0000DDFFF7E7EC1400201815002080
:104D0C0010B5094B1B68191F1A680B689A4208D119
:104D1C00064A136802331360034A1368043B13609A
:104D2C0010BDFFF7C5FFF7E7EC14002018150020A5
:104D3C0010B5094B1B68191F1A680B689A4208DDDD
:104D4C00064A136802331360034A1368043B13606A
:104D5C0010BDFFF7ADFFF7E7EC140020181500208D
:104D6C0010B5094B1B68191F1A680B689A4208DAB0
:104D7C00064A136802331360034A1368043B13603A
:104D8C0010BDFFF795FFF7E7EC1400201815002075
:104D9C0030B589B001A80E4B020032CB32C232CBF7
:104DAC0032C21B88138000F0C0FFFCF709F8002802
:104DBC00FBD0FF231840592805D0064800F0B5FF5A
:104DCC00002009B030BD0D20FBF796FD0120F8E75F
:084DDC00905E0008F455000888
:104DE400F0B58FB0040001A9394B0A0023CB23C2CC
:104DF40023CB23C223CB23C203CB03C2354B1B6873
:104E04005F2B12D0344D354E33682B60FDF782FB97
:104E140033682B60FDF71EFC051E10D0304A80233A
:104E240011680B431360002506E02D4A8023DB0044
:104E340011680B431360002528000FB0F0BDFDF787
:104E440077FC002804D10CA801002A00254F0EE0AD
:104E540001A800F06EFFFFF79FFF0028F3D10225A1
:104E6400EAE7002B12D0072A0AD001320131D35DC0
:104E74000B701E00613E192EF3D8203B0B70F2E735
:104E8400174A022311680B431360D5E70CAB1B7858
:104E9400002B0CD00F4A12681201134952185355B3
:104EA40001354378002B02D00130072DF7D1094B8F
:104EB4001A6812010C4B9B185D1900226A700B4A88
:104EC40010680B4A82189A602043D8600125B3E722
:104ED400A855000808150020AC140020B8140020C0
:104EE400241500205C140020040800203415002040
:044EF4000402002094
:104EF80070B5C0200005FFF771FF00280DD00A4CDF
:104F080022680A4803681D010949491915688D6016
:104F1800043A22600133036070BD064A8023116899
:104F28000B431360F8E7C046EC1400200815002076
:084F38000408002024150020EC
:104F400010B50020FFF74EFF002808D0022807D038
:104F5000074B1A68074B1A60074B01221A6010BDF5
:104F6000064B1B681B01064A00219954F7E7C0460F
:104F700034150020301500202815002008150020C9
:044F80000408002001
:104F840010B51A4A13681C68043B1360022C1AD823
:104F9400002821D1164800F0CCFE164800F0C9FEC6
:104FA40020003030C0B2FBF7ABFC002C18D020201E
:104FB400FBF7A6FC3F20FBF7A3FCFFF7EDFE002860
:104FC40012D0200010BD0C4A8023DB0011680B4373
:104FD400136001246442F4E7084800F0AAFEDCE709
:104FE400074800F0A6FEE2E70324EAE7EC140020F9
:104FF400C05F0008D45F000824150020F05F00089B
:04500400A05F0008A1
:1050080010B50120FFF7BAFF022800D910BD054CE2
:105018002060FBF737F92368002BF7D0FBF7D2F9AC
:08502800F4E7C0465C1500200E
:1050300010B50020FFF7A6FF02280AD8074B18601A
:10504000002807D1FFF726FDFBF7E4F8034B002209
:105050001A6010BDFBF774FCFBE7C0465C1500202E
:10506000074B1B68002B09D0054B00221A60054A2C
:105070001368191D1160044A12685A607047C046CF
:0C50800040150020EC1400203C1500201E
:10508C0010B5214B1A68214B1A60FDF73FFAFDF75A
:10509C0087FB002821D01C4B1A681C4B1A601C4B38
:1050AC001A6812011B4B9B18DA68C0231B051A42A5
:1050BC0019D0194B1B68002B1BD1184B1B68002BEC
:1050CC001AD117480368124A11680901114A52187B
:1050DC0019689160043B036004E0124AA023116834
:1050EC000B43136010BD0F4A802311680B431360F0
:1050FC00F8E7FFF7AFFFE0E76920FDF7BBFB044BD8
:10510C001868FDF7B7FBEDE7B8140020AC140020CD
:10511C00FC14002004080020201500202815002075
:08512C00EC1400202415002002
:1051340010B5094B1B68002B0BD1084A13680849AA
:1051440018680860043B1360FDF7D6FEFDF74AFFBC
:1051540010BDFFF783FFF0E720150020EC140020BA
:0451640038150020DA
:1051680010B5114B1B68002B0DD1104A136810495C
:1051780018680860043B13600E4B1B88DB0705D5D5
:10518800FDF72EFF10BDFFF767FFEEE70A4B1E2263
:105198001A600A4B1968F020400000F0C3FF084B62
:1051A8001860FDF7A7FEEBE720150020EC1400209F
:1051B800001500200004004038150020E4140020E9
:0451C8001C15002092
:1051CC0010B5344B1B68002B2FD1334B9B6C013328
:1051DC002ED0324B1B68002B0DD1314A1360314A53
:1051EC0013609023DB051A680F218A431A601A6832
:1051FC000A390A431A602C490B681A68274802605E
:10520C00043B0B60002A0AD19023DB05802252025A
:10521C009A61802292029A611F4B00229A64214B60
:10522C0000221A60FDF734FF10BDFFF713FFCCE727
:10523C001A4B00221A609023DB051A680F218A434F
:10524C001A601A680A390A431A60174B1A681368ED
:10525C00002B09DD9023DB05802252029A61022289
:10526C009A61FFF77BFFDFE7002B08DB9023DB0560
:10527C00802252029A61802292029A61F1E75B428B
:10528C0013609023DB0501229A61802292029A61BD
:10529C00E7E7C0462015002004080020D0140020A9
:0C52AC00D4140020E8140020EC140020B2
:1052B800F0B5C64600B588B069462B4B0A0013CB3B
:1052C80013C213CB13C203CB03C2284B1B68002B9A
:1052D80014D1274A13688024A40519680C43043B99
:1052E8001360244B9C420CD9234A8023DB001168AD
:1052F8000B43136008B080BCB846F0BDFFF7ACFEA6
:10530800E7E70D20FBF7FAFA684600F010FD2000E9
:1053180000F082FE270080370F25032398460FE010
:105328000D20FBF7EBFA200000F076FE3A20FBF7A1
:10533800E5FA300000F025FD00250134BC420ED00E
:1053480026780135102DEBD0300000F01AFD4346C9
:105358002B40032BF1D17C20FBF7D0FAEDE70D2091
:10536800FBF7CCFAC6E7C046D45500082015002044
:0C537800EC140020807F00202415002091
:1053840010B5214B1B68002B34D1204B1B681A68C5
:10539400012A32D9012200241D490A60043B1B4919
:1053A4000B601C4B5868F0218843586059682143AE
:1053B400596053019B1A99008918C900164B186843
:1053C40000F0B2FE013880235B0498420DD2134AE8
:1053D40050601348036A1B021B0AC02109060B43D1
:1053E400036200239360073313600E4B1B68002B8A
:1053F40006D110BDFFF732FEC7E71022B024CBE779
:10540400FDF77AFDF5E7C04620150020EC140020D6
:10541400E4140020001002400002002010E000E02C
:0854240000ED00E01C15002062
:10542C00114B1A6801210A431A605A680F4802404E
:10543C005A601A680E4802401A601A680D480240F9
:10544C001A605A680C4802405A60DA6A0F2082438C
:10545C00DA621A6B094802401A635A6B8A435A6320
:10546C0000229A607047C046001002400CB8FFF84A
:10547C00FFFFF6FEFFFFFBFFFFFFC0FFACFEFFFFD1
:10548C00074B1B68002B00DBFEE7054A11688023E5
:10549C001B060B4313608369023383617047C0465C
:0454AC002CED00E003
:1054B00020286329323032302D323420572E536366
:0854C00068656D6D65727400F2
:0854C8004B65726E656C3A0041
:1054D000537461636B3D0000436F6465546872658B
:1054E00061643D00456D7074795F000050726F6AB1
:1054F0006563740020204155544F4558453D0000D8
:105500002020204C45446D6F64653D0020202043E1
:105510005055636C6F636B3D000000004261756421
:10552000526174653D0000002870656E64696E67A5
:10553000290000002020465245513D00487A205065
:10554000574D313D000000002020204D4F543A00BF
:10555000537465703D0000006D73204E5354503DF0
:0C5560000000000044432F50574D310064
:10556C00416374697665206174206E65787420538C
:0C557C00797374656D20537461727400C3
:105588004C380008A2380008B4380008C6380008AB
:10559800D8380008EA380008FC380008283900081C
:1055A800205761726E3A2077696C6C206F7665724D
:1055B80072696465204B65726E656C204F50207768
:0C55C8002E73616D65206E616D65200022
:1055D400313238205352414D2062797465732073FF
:1055E40074617274696E672066726F6D2030780022
:0C55F4002063616E63656C6C65642000D0
:10560000000000000000000000000000000000009A
:10561000000000000000000000000000000000008A
:10562000000000000000000000000000000000007A
:10563000000000000000000000000000000000006A
:10564000000000000000000000000000000000005A
:10565000000000000000000000000000000000004A
:10566000000000000000000000000000000000003A
:10567000000000000000000000000000000000002A
:10568000000000000000000000000000000000001A
:105690000000000000000000000001000000050004
:1056A00000000000000000000000000000000000FA
:1056B00000000000000000000000000000000100E9
:1056C00000000400000004000000000000000000D2
:1056D00000000000000000000000000000000000CA
:1056E00000000400000004000000040000000000AE
:1056F00000000000000000000000000000000000AA
:105700000000000000000000000000000000000099
:10571000000004000000000000000500000005007B
:105720000000050000000400000004000000040068
:105730000000040000000000000001000000010063
:105740000000010000000100000003000000030051
:10575000000003000000030000000300000003003D
:10576000000003000000030000000300000003002D
:10577000000003000000030000000200000002001F
:105780000000020000000200000002000000010012
:1057900000000100000008000000080000000800F0
:1057A00000000800000008000000080000000800D9
:1057B00000000800000008000000080000000800C9
:1057C00000000800000008000000080000000800B9
:1057D00000000800000002000000020000000100BC
:1057E00000000100000000000000040000000500AF
:0857F0000000010000000100AF
:1057F8004552524F5200000044524F5000000000E2
:10580800445550000000000053574150000000006C
:105818004F56455200000000524F5400000000004F
:105828002D524F54000000005049434B0000000027
:10583800524F4C4C00000000494E4A45435400006A
:105848002B00000000000000312B000000000000C9
:105858002D00000000000000312D000000000000B5
:1058680041425300000000005348494654000000DC
:10587800414E4400000000004F52000000000000AC
:10588800584F5200000000004E4F54000000000026
:105898002B2F2D00000000002A000000000000004F
:1058A8002F000000000000002A2F00000000000068
:1058B8004D4F4400000000002F4D4F4400000000F1
:1058C800425345540000000042434C52000000007F
:1058D800425453540000000052414E444F4D0000C2
:1058E8003D3D000000000000213D000000000000D8
:1058F8003E000000000000003E3D000000000000E7
:105908003C00000000000000553C000000000000C2
:105918003C3D000000000000303D00000000000099
:10592800564152434F4E00005245560000000000B9
:1059380041525241590000004B45593F00000000B8
:105948004B45590000000000454D49540000000037
:105958002E000000000000002E480000000000009B
:105968002E440000000000002E220000000000006D
:10597800445A0000000000004858000000000000E1
:10598800584E4F50000000004D530000000000002A
:105998004453000000000000544958000000000073
:1059A80054494D4500000000534C45455000000047
:1059B800465245510000000050574D31000000008C
:1059C8004D4F5400000000004F4800000000000048
:1059D8004F4C000000000000495055000000000036
:1059E8004950440000000000495A0000000000002F
:1059F8005244494E00000000524144430000000058
:105A0800494E492D535049005350490000000000A9
:105A18002E53000000000000465300000000000064
:105A28004F5053000000000055534552000000003D
:105A380053454500000000004D454D0000000000A2
:105A4800535400000000000052554E0000000000B2
:105A58004E4F2D4442470000444542554700000040
:105A6800464F52474554000041424F5254000000EF
:105A78005245504C41434500524553544F524500FE
:105A88004946000000000000434153450000000063
:105A98003C434153450000003E434153450000004C
:105AA800454C5345000000005448454E0000000096
:105AB800444F000000000000554E54494C000000BF
:105AC8005748494C45000000414741494E000000F5
:105AD800464F5200000000004C4F4F50000000009D
:105AE8004900000000000000434F4E5449000000E8
:105AF800425245414B0000005A425245414B00007A
:105B080052455455524E00003A0000000000000073
:105B18003B00000000000000646F53545200000076
:105B2800646F4C4954384200646F4C49540000007B
:105B3800646F56414C554500646F5245560000004D
:105B4800646F494600000000646F434153450000FC
:105B5800646F3C4341534500646F3E4341534500E5
:105B6800646F454C53450000646F444F00000000CB
:105B7800646F554E54494C00646F5748494C450072
:105B8800646F414741494E00646F464F5200000020
:105B9800646F4C4F4F50000052502D3100000000F0
:105BA80052502D34000000004155544F45584500CF
:105BB80042415544000000004C45440000000000EC
:105BC80053504545440000003F000000000000001D
:105BD80053415645000000004C4F4144000000006E
:105BE800FEE7FEE7FEE7FEE7FEE7FEE7FEE7FEE785
:105BF800FEE7FEE7FEE7FEE7FEE7FEE7FEE7FEE775
:105C0800FEE7FEE7FEE7FEE7FEE7FEE7FEE7FEE764
:105C1800FEE7FEE7FEE7FEE7FEE7FEE7FEE7FEE754
:105C2800FEE7FEE7FEE7FEE7FEE7FEE7FEE7FEE744
:105C3800FEE703488546FFF7F5FB03E070470000E1
:045C48000018002020
:105C4C0011488546114C20680434004201D080472D
:105C5C00F9E70F480F49091A082903DB00220260F3
:105C6C00043001600C480D49884205D002680430AC
:105C7C0003B4904703BCF7E700208646EC460020AF
:105C8C000021074A9047FEE70018002094610008A5
:105C9C0078150020C0160020E95E0008E95E0008B7
:045CAC00550C00088B
:105CB00004207146084202D1EFF3088001E0EFF3BF
:0C5CC00009800149084700008D540008CD
:105CCC0043466F727468204C6F77506F7765722DF6
:105CDC0034384D487A2F334D487A2C6E6F555342D9
:105CEC002D20666F722053544D333246303432209F
:025CFC00760030
:0A5CFE003323013B002BFCD170475B
:105D0800756E646572666C6F77212000202D2D2DCD
:025D1800200069
:105D1A0010B502003030C0B2392801D93732D0B2BA
:065D2A00FAF7EBFD10BDCD
:065D30002849502D3E0041
:105D360010B5441C0078002806D0FAF7E0FD0134BF
:0A5D4600631E18780028F8D110BD84
:105D500063616E277420534545204B65726E656CF8
:105D6000204F7073000000005573657248656164D0
:105D700065725F5374727563743D000056617243BF
:0A5D80006F6E3A56616C75653D00C8
:105D8A0010B5040003061B0F18003030392801D95A
:105D9A0037331800FAF7B1FD0F20044020003030E5
:105DAA00392800D90730FAF7A8FD2020FAF7A5FD0F
:025DBA0010BD1A
:105DBC004572726F722300002028636F6C20000004
:105DCC00206E6F7420666F756E6400005F53796E81
:105DDC0074617820457272005F537461636B204567
:105DEC00727200005F436F6D70696C65206F6E6C32
:105DFC00790000005F496E76616C696420436F64C2
:105E0C006520616363657373000000005F6F7574D8
:105E1C00206F6620436F6E74657874005F52756EE8
:105E2C0074696D65206F6E6C790000005F54687248
:105E3C006561642063616E63656C6C656400000071
:105E4C005F4E756D626572206F7574206F6620529F
:105E5C00616E6765000000005F4469762E627920F0
:105E6C005A65726F000000002020636F6D70696CC2
:065E7C00696E672E2E0086
:0E5E820010B5FAF718FE2020FAF73BFD10BD10
:105E900020636F6E6669726D20772E757070657203
:0A5EA0002063617365202759270075
:105EAA002F280FD90300303BDBB2092B08D90A2966
:105EBA000BD00300413B052B0AD83738C0B27047D4
:105ECA001800FCE701204042F9E701204042F6E7CA
:065EDA0001204042F3E745
:095EE00028566172436F6E3D000B
:0E5EEA0010B56A20FCF7C7FCFDF735FE10BDB1
:105EF800203C2D6E6F742061204B65726E656C209E
:105F08004F50206E6F722061206E756D6265720051
:105F1800203C2D696E76616C696420666F72204240
:105F280061636B2D4374726C00000000203C2D529D
:0D5F3800756E74696D65204572726F7200A0
:0E5F460010B56B20FCF799FCFDF707FE10BDAF
:105F540020202841444320696E69742920000000F0
:0D5F6400202028414443206F66662920005C
:0E5F720010B56C20FCF783FCFDF7F1FD10BDAF
:105F80002064656275672066696E69736865642060
:015F90000010
:0E5F920010B56D20FCF773FCFDF7E1FD10BDAE
:105FA000283D456D7074792050726F6A656374295D
:015FB00000F0
:0E5FB20010B57020FCF763FCFDF7E5FD10BD97
:055FC0004C6F6164005C
:0E5FC60010B57120FCF759FCFDF7DBFD10BD96
:0D5FD4002050726F6A656374206E6F2E009E
:0E5FE20010B57220FCF74BFCFDF7CDFD10BD95
:055FF00053617665001D
:105FF6000A0010D00300400800E052008242FCD99B
:10600600002000E05208934200D39B1A40418A4286
:0A601600F8D1190070470020704710
:1060200070B50400000FFFF778FE200E0F25284002
:10603000FFF773FE200D2840FFF76FFE200C28406D
:10604000FFF76BFE200B2840FFF767FE200A284071
:10605000FFF763FE20092840FFF75FFE280020407D
:0C606000FFF75BFE2020FAF74DFC70BD3E
:10606C0010B50400000F16D12001000F17D120022B
:10607C00000F18D12003000F19D12004000F1AD1E2
:10608C002005000F1BD12006000F1CD10F20204033
:10609C00FFF73DFE10BDFFF73AFE2001000FFFF7A2
:1060AC0036FE2002000FFFF732FE2003000FFFF731
:1060BC002EFE2004000FFFF72AFE2005000FFFF72D
:0C60CC0026FE2006000FFFF722FEDFE793
:1060D80010B504003020FAF711FC7820FAF70EFC0E
:0860E8002000FFF7BFFF10BD0F
:1060F000CA1751408B1A17D0C1174A4004B4484000
:10610000411A48081A0000E052008242FCD90020DF
:1061100000E05208914200D3891A40419A42F8D1D6
:0C61200004BC5040801A704700207047FB
:10612C000A000FD00300400800E052008242FCD964
:10613C00002000E05208934200D39B1A40418A424F
:08614C00F8D1704700207047F4
:10615400CA1751408B1A19D0C11706B44840411AC6
:1061640048081A0000E052008242FCD9002000E0F6
:106174005208914200D3891A40419A42F8D10CBC8A
:1061840053405840C01A5140891A70470020704744
:10619400B96300080402002071130000CF630008F3
:1061A40000000020B46100080402000000000000A8
:1061B400150F0008250F00084D0F00087D0F00087B
:1061C400950F0008A90F0008CD0F0008F10F000873
:1061D4003110000891100008F11000080D1100089A
:1061E4001D11000839110008491100086111000847
:1061F400A9110008C5110008E1110008FD110008EB
:106204000D1200081D12000839120008711200084E
:10621400A9120008E112000821130008591300080C
:1062240091130008CD130008E513000805140008B5
:10623400391400085D14000881140008A51400082E
:10624400C514000825140008F94E00088D500008F4
:10625400E91400082D2D00089D1A0008111A0008E1
:10626400F91A0008411B0008291D0008152E000812
:106274003D1500085D1500087D150008CD310008A6
:106284007D32000899150008B5150008E5360008A8
:106294003551000869510008CD510008B932000891
:1062A4006533000815340008B93400085D3500086A
:1062B400ED350008C9370008ED390008293A00080F
:1062C400611B0008D1160008411D0008251C0008A8
:1062D400F5420008B9520008F1160008FD1600083E
:1062E40009170008291A0008894600080147000810
:1062F400E14B00086D4C0008EB5E0008475F0008A6
:10630400735F0008935F0008652A0008D51500082C
:10631400AD2A0008B35F0008C75F0008E35F000808
:10632400D92A0008052B000809160008451800089A
:10633400251600083916000861160008414F0008A8
:106344005D2B00086D1A0008551700081517000882
:1063540075170008A1170008E14C00080D4D00084E
:106364003D4D00086D4D0008CD170008F1170008D9
:1063740075180008AD18000821180008E518000871
:1063840035190008C1190008D11900082928000886
:1063940095220008E119000885530008D91D00085A
:1063A40009500008315000080100000014130020B7
:0463B400006CDC029B
:1063B800206861680834094204D000220270013064
:0663C8000139FBD1704712
:1063CE0020686168A2680C34124205D00B78037005
:0A63DE0001300131013AF9D1704796
:0400000508005C3B58
:00000001FF
